:103800000C942A1C0C94451C0C94451C0C94451CCF
:103810000C94451C0C94451C0C94451C0C94451CA4
:103820000C94451C0C94451C0C94451C0C94451C94
:103830000C94451C0C94451C0C94451C0C94451C84
:103840000C94451C0C94451C0C94451C0C94451C74
:103850000C94451C11241FBECFE5D4E0DEBFCDBFC4
:1038600010E0A0E6B0E0EAEAFCE302C005900D92A9
:10387000A036B107D9F710E0A0E6B0E001C01D9274
:10388000A33EB107E1F70C945D1C0C94001C81E48D
:103890000E94221E86E50E94221E82E50E94221EB0
:1038A00082E40E94221E8FE40E94221E8FE40E9466
:1038B000221E84E50E94221E0895CFE5D4E0DEBFDB
:1038C000CDBF81E085BF82E085BF60E087E190E009
:1038D0000E94181E0E94371E682F813611F489E558
:1038E000C3C08134A9F40E94371E99279093E10048
:1038F0008093E000182F00270E94371E9927082B7D
:10390000192B000F111F1093E1000093E00052C02B
:10391000823641F489E50E94221E80E00E94221E28
:1039200080E8A2C0823489F40E94371E9927182F9C
:1039300000270E94371E9927082B192B0E94371E3B
:10394000682FC8010E94371D8FC0873689F40E94F6
:10395000371E9927182F00270E94371E9927082BFA
:10396000192B0E94371E682FC8010E94D61DB2CFA6
:10397000853611F58091E2008537C1F41092E1009F
:103980001092E00020E030E083E0F90180935700DE
:10399000E89507B600FCFDCF20583F4F88E3203064
:1039A000380790F33093E1002093E00081E18093A9
:1039B0005700E8958DE058C0853451F488E190E0D7
:1039C00028E00FB6F894A89581BD0FBE21BDF2CFB7
:1039D000803581F38C3471F3803711F483E544C072
:1039E000863421F469E080E090E005C0823731F44C
:1039F00069E081E090E00E944B1E36C08E3421F4D5
:103A000069E083E090E0F7CF813569F1843729F4EC
:103A100085E70E94221E80E027C08857823018F474
:103A20000E94371EC7CF643529F40E94371E809349
:103A3000E200C0CF633519F40E94471C4BCF6635B6
:103A400029F480E30E94221E84E30EC0633741F410
:103A500083E00E94221E84E90E94221E8EE104C09F
:103A60006B3109F437CF8FE30E94221E33CFDF92F0
:103A7000EF92FF920F931F93CF93DF938C01D62E7B
:103A800060E070E0EB01C05ADF4F7B010894E11C5D
:103A9000F11C6017710718F40E94371E01C08FEFE8
:103AA0008883B7016038710568F360E070E0C09109
:103AB000E000D091E1008CB399279C012270307016
:103AC00081FDF9CF8091E200853709F066C0FFB62D
:103AD000F89486E4D81609F03EC04091E000509179
:103AE000E100DB01A05ABF4F8D91282F33278D9124
:103AF0009927982F8827282B392B6E5F7F4F81E0DD
:103B00000901FA0180935700E89511244E5F5F4F39
:103B10000250104049F75093E1004093E000C07814
:103B200085E0FE0180935700E89507B600FCFDCFC5
:103B300081E180935700E8958091E0009091E10049
:103B40009C0120788217930731F020583F4F309323
:103B5000E1002093E00085E4D816D9F4FB01E05A97
:103B6000FF4F8091E0008EBB8091E0009091E100DA
:103B7000292F33272FBB01969093E1008093E0001B
:103B800081918DBBE29AE19AE199FECF01501040FC
:103B900041F7FFBE8DE090E001C0C901DF91CF91F8
:103BA0001F910F91FF90EF90DF900895FF920F9378
:103BB0001F93CF93DF93EC01FFB6F894E199FECF0A
:103BC0006534B1F48091E0008EBB8091E00090916B
:103BD000E100292F33272FBB01969093E1008093BA
:103BE000E000E09A8DB30E94221E219759F719C078
:103BF00060E08091E0009091E1000E944B1E8C01FA
:103C00000E94221E812F99270E94221E8091E0008F
:103C10009091E10002969093E1008093E00022975A
:103C200039F7FFBEDF91CF911F910F91FF9008955B
:103C30009C01832F992780BD29B988E18AB986E83C
:103C400080BD089520E030E08CB90FB607FE0BC0B0
:103C50005E990BC02F5F3F4F5E9907C087E220310E
:103C60003807C4F302C05E9BFECF5E9A089580E0E1
:103C700090E00FB607FE0AC05F990AC001965F99EF
:103C800007C027E280319207CCF302C05F9BFECFD2
:103C90008CB199270895FC0160FD60935700C89589
:0A3CA000802DE395C895902D08953E
:0400000300003800C1
:00000001FF
